******************************************************************************
            TI ARM Clang Linker PC v1.3.0                      
******************************************************************************
>> Linked Thu Nov 17 12:12:46 2022

OUTPUT FILE NAME:   <D:/TI_SITARA/MCAL_AM263x_00.09.00_03/mcal/binary/can_app/bin/am263/can_app_r5f_release.xer5f>
ENTRY POINT SYMBOL: "_c_int000"  address: 00000000


MEMORY CONFIGURATION

         name            origin    length      used     unused   attr    fill
----------------------  --------  ---------  --------  --------  ----  --------
PAGE 0:
  RESET_VECTORS         00000000   00000100  00000068  00000098     X
  TCMA_RAM              00000100   00003f00  00000120  00003de0  R  X
  TCMB_RAM              00080000   00004000  00000000  00004000  RW  
  VECTORS               102ef000   00001000  00000000  00001000     X
  HWA_RAM               28000000   00020000  00000000  00020000  RW  
  L2_RAM_BANK0          70080000   00100000  0001a2de  000e5d22  RW  
  L3_RAM                88000000   00300000  00000000  00300000  RW  

PAGE 1:
  L3_RAM                88000000   00300000  00000000  00300000  RW  


SEGMENT ALLOCATION MAP

run origin  load origin   length   init length attrs members
----------  ----------- ---------- ----------- ----- -------
00000000    00000000    00000068   00000068    r-x
  00000000    00000000    00000068   00000068    r-x .intvecs
00000100    00000100    00000120   00000120    r-x
  00000100    00000100    00000120   00000120    r-x .startup
70080000    70080000    00007994   00007994    r-x
  70080000    70080000    00007994   00007994    r-x .text
70087998    70087998    00004998   00000000    rw-
  70087998    70087998    00004998   00000000    rw- .bss
7008c330    7008c330    00004000   00002000    rw-
  7008c330    7008c330    00002000   00002000    rw- .stack
  7008e330    7008e330    00002000   00000000    rw- .sysmem
70090330    70090330    00006be0   000037e0    r--
  70090330    70090330    00001dde   00001dde    r-- .rodata
  70092110    70092110    00001a00   00001a00    r-- McalConstSection
  70093b10    70093b10    00001a00   00000000    r-- McalInitSection
  70095510    70095510    00001a00   00000000    r-- McalNoInitSection
70096f10    70096f10    00001a00   00001a00    r--
  70096f10    70096f10    00001a00   00001a00    r-- McalTextSection
70098910    70098910    00001320   00000000    rw-
  70098910    70098910    00001320   00000000    rw- .data
70099c30    70099c30    000006b4   000006b4    r--
  70099c30    70099c30    00000200   00000200    r-- .const
  70099e30    70099e30    000004b4   000004b4    r-- .cinit


SECTION ALLOCATION MAP

 output                                  attributes/
section   page    origin      length       input sections
--------  ----  ----------  ----------   ----------------
.intvecs   0    00000000    00000068     
                  00000000    00000038     sys_intvecs.oer5f (.intvecs)
                  00000038    00000008     sys_startup.oer5f (.tramp._sysResetEntry_.1)
                  00000040    00000008     sys_startup.oer5f (.tramp._sysUndefEntry_.1)
                  00000048    00000008     sys_startup.oer5f (.tramp._sysSvcEntry_.1)
                  00000050    00000008     sys_startup.oer5f (.tramp._sysPrefetchEntry_.1)
                  00000058    00000008     sys_startup.oer5f (.tramp._sysDAbortEntry_.1)
                  00000060    00000008     sys_startup.oer5f (.tramp._sysIrqEntry_.1)

.startup   0    00000100    00000120     
                  00000100    00000088     app_utils.aer5f : sys_vim.oer5f (.startup.vimIrqDispatcher)
                  00000188    00000008     --HOLE-- [fill = 0]
                  00000190    00000084                     : sys_vim.oer5f (.startup.vimFiqDispatcher)
                  00000214    0000000c     --HOLE-- [fill = 0]

.text      0    70080000    00007994     
                  70080000    00000100     --HOLE-- [fill = feaa55ef]
                  70080100    000011de     can.aer5f : Can_Mcan.oer5f (.text:CAN_TEXT_SECTION)
                  700812de    00000002     --HOLE-- [fill = 0]
                  700812e0    00000ed0     libc.a : _printfi.c.obj (.text:__TI_printfi)
                  700821b0    00000c58     can.aer5f : mcan.oer5f (.text:CAN_TEXT_SECTION)
                  70082e08    00000008     libc.a : pre_init.c.obj (.text._system_pre_init)
                  70082e10    00000ab6     mcu.aer5f : Mcu_Platform.oer5f (.text:MCU_TEXT_SECTION)
                  700838c6    00000002     --HOLE-- [fill = 0]
                  700838c8    00000008     libc.a : exit.c.obj (.text:abort)
                  700838d0    0000097e     can.aer5f : Can.oer5f (.text:CAN_TEXT_SECTION)
                  7008424e    00000002     --HOLE-- [fill = 0]
                  70084250    00000520     CanApp.oer5f (.text.CanExample_ExternalTest)
                  70084770    00000458     mcu.aer5f : Mcu.oer5f (.text:MCU_TEXT_SECTION)
                  70084bc8    00000008     libc.a : copy_decompress_rle.c.obj (.text:decompress:rle24)
                  70084bd0    00000404     port.aer5f : Port.oer5f (.text:PORT_TEXT_SECTION)
                  70084fd4    000003b0     sys_startup.oer5f (.text)
                  70085384    0000000c     libc.a : aeabi_portable.c.obj (.text.__aeabi_errno_addr)
                  70085390    000002ec     port.aer5f : Port_Platform.oer5f (.text:PORT_TEXT_SECTION)
                  7008567c    00000004     libc.a : mpu_init.c.obj (.text.__mpu_init)
                  70085680    00000278            : _printfi.c.obj (.text._pconv_a)
                  700858f8    00000004     libclang_rt.builtins.a : aeabi_memcpy.S.obj (.text)
                  700858fc    00000004     --HOLE-- [fill = 0]
                  70085900    00000264     can.aer5f : Can_Priv.oer5f (.text:CAN_TEXT_SECTION)
                  70085b64    00000004     --HOLE-- [fill = 0]
                  70085b68    00000230     libc.a : _printfi.c.obj (.text._pconv_g)
                  70085d98    00000008     --HOLE-- [fill = 0]
                  70085da0    000001d0     can.aer5f : Can.oer5f (.text:CAN_ISR_TEXT_SECTION)
                  70085f70    000001d0     libclang_rt.builtins.a : udivsi3.S.obj (.text)
                  70086140    0000017c     CanApp.oer5f (.text.main)
                  700862bc    0000016e     app_utils.aer5f : sys_core.oer5f (.text)
                  7008642a    00000006     --HOLE-- [fill = 0]
                  70086430    00000148     libc.a : _printfi.c.obj (.text.fcvt)
                  70086578    00000140            : s_scalbn.c.obj (.text.scalbn)
                  700866b8    00000130            : _printfi.c.obj (.text._pconv_e)
                  700867e8    00000118     libclang_rt.builtins.a : udivmoddi4.S.obj (.text)
                  70086900    000000d2     app_utils.aer5f : sci.oer5f (.text.sciAInit)
                  700869d2    00000002     --HOLE-- [fill = 0]
                  700869d4    000000bc     libc.a : _printfi.c.obj (.text._mcpy)
                  70086a90    000000b8            : copy_decompress_rle.c.obj (.text.__TI_decompress_rle_core)
                  70086b48    00000088            : _ltoa.c.obj (.text.__TI_ltoa)
                  70086bd0    00000088            : _printfi.c.obj (.text._ecpy)
                  70086c58    0000007c            : s_frexp.c.obj (.text.frexp)
                  70086cd4    00000074            : _printfi.c.obj (.text._pconv_f)
                  70086d48    00000008     --HOLE-- [fill = 0]
                  70086d50    00000074     can.aer5f : Can_Irq.oer5f (.text:CAN_ISR_TEXT_SECTION)
                  70086dc4    0000000c     CanApp.oer5f (.tramp.main.1)
                  70086dd0    0000006c     CanApp.oer5f (.text.CanIf_RxIndication)
                  70086e3c    0000006c     libc.a : atoi.c.obj (.text.atoi)
                  70086ea8    00000008     --HOLE-- [fill = 0]
                  70086eb0    00000068     app_utils.aer5f : sys_vim.oer5f (.text.vimRegisterInterrupt)
                  70086f18    00000008     --HOLE-- [fill = 0]
                  70086f20    00000064                     : sys_vim.oer5f (.text.vimInit)
                  70086f84    00000064     libc.a : vsnprintf.c.obj (.text.vsnprintf)
                  70086fe8    0000005c            : autoinit.c.obj (.text:__TI_auto_init_nobinit_nopinit)
                  70087044    00000058            : _printfi.c.obj (.text._fcpy)
                  7008709c    00000058            : vsnprintf.c.obj (.text._outs)
                  700870f4    0000000c     can.aer5f : Can.oer5f (.tramp.Can_3_Int1ISR_Fun.1)
                  70087100    00000058     app_utils.aer5f : sci.oer5f (.text.sciSend)
                  70087158    00000008     --HOLE-- [fill = 0]
                  70087160    00000056                     : trace.oer5f (.text.GT_trace1)
                  700871b6    00000002     --HOLE-- [fill = 0]
                  700871b8    00000054     libc.a : boot_non_cortex_m.S.obj (.text)
                  7008720c    00000004     --HOLE-- [fill = 0]
                  70087210    00000052     app_utils.aer5f : trace.oer5f (.text.GT_trace0)
                  70087262    00000002     --HOLE-- [fill = 0]
                  70087264    0000000c     can.aer5f : Can.oer5f (.tramp.Can_3_Int0ISR_Fun.1)
                  70087270    0000004a     app_utils.aer5f : sys_vim.oer5f (.text.vimInterruptsInit)
                  700872ba    00000002     --HOLE-- [fill = 0]
                  700872bc    00000048     libc.a : memccpy.c.obj (.text.memccpy)
                  70087304    0000000c     can.aer5f : Can.oer5f (.tramp.Can_2_Int1ISR_Fun.1)
                  70087310    00000044     app_utils.aer5f : sci.oer5f (.text.sciReceive)
                  70087354    0000000c     can.aer5f : Can.oer5f (.tramp.Can_2_Int0ISR_Fun.1)
                  70087360    0000003a     app_utils.aer5f : app_utils.oer5f (.text.AppUtils_defaultInit)
                  7008739a    00000006     --HOLE-- [fill = 0]
                  700873a0    0000003a                     : app_utils.oer5f (.text.AppUtils_printf)
                  700873da    00000006     --HOLE-- [fill = 0]
                  700873e0    00000036                     : app_utils.oer5f (.text.AppUtils_getStackUsage)
                  70087416    0000000a     --HOLE-- [fill = 0]
                  70087420    00000036                     : app_utils_uart.oer5f (.text.message)
                  70087456    0000000a     --HOLE-- [fill = 0]
                  70087460    00000036                     : sci.oer5f (.text.sciDisableNotification)
                  70087496    00000002     --HOLE-- [fill = 0]
                  70087498    00000030     libc.a : vsnprintf.c.obj (.text._outc)
                  700874c8    00000008     --HOLE-- [fill = 0]
                  700874d0    0000002c     Dem.oer5f (.text.Dem_SetEventStatus)
                  700874fc    00000004     --HOLE-- [fill = 0]
                  70087500    0000002c     libclang_rt.builtins.a : divsi3.S.obj (.text)
                  7008752c    00000004     --HOLE-- [fill = 0]
                  70087530    0000002a     CanApp.oer5f (.text.GT_assertLocal)
                  7008755a    00000002     --HOLE-- [fill = 0]
                  7008755c    00000028     libc.a : _printfi.c.obj (.text.strchr)
                  70087584    00000024     libclang_rt.builtins.a : aeabi_uldivmod.S.obj (.text)
                  700875a8    00000008     --HOLE-- [fill = 0]
                  700875b0    00000020     CanApp.oer5f (.text.CanIf_ControllerModeIndication)
                  700875d0    00000020     CanApp.oer5f (.text.Det_ReportError)
                  700875f0    00000020     libc.a : args_main.c.obj (.text._args_main)
                  70087610    00000020            : wcslen.c.obj (.text.wcslen)
                  70087630    0000001c     app_utils.aer5f : app_utils.oer5f (.text.AppUtils_getChar)
                  7008764c    00000004     --HOLE-- [fill = 0]
                  70087650    0000001c     CanApp.oer5f (.text.CanIf_TxConfirmation)
                  7008766c    0000001c     libc.a : _printfi.c.obj (.text.strlen)
                  70087688    0000001c     libsysbm.a : memcpy32.S.obj (.text:TI_memcpy_small)
                  700876a4    0000001c     libclang_rt.builtins.a : aeabi_memset.S.obj (.text)
                  700876c0    0000001a     app_utils.aer5f : sci.oer5f (.text.sciSetBaudrateValue)
                  700876da    00000002     --HOLE-- [fill = 0]
                  700876dc    00000018     libsysbm.a : memset32.S.obj (.text:TI_memset_small)
                  700876f4    0000000c     can.aer5f : Can.oer5f (.tramp.Can_1_Int1ISR_Fun.1)
                  70087700    00000016     CanApp.oer5f (.text.Dem_ReportErrorStatus)
                  70087716    0000000a     --HOLE-- [fill = 0]
                  70087720    00000016     app_utils.aer5f : app_utils_uart.oer5f (.text.Enable_Uart)
                  70087736    0000000a     --HOLE-- [fill = 0]
                  70087740    00000014                     : app_utils.oer5f (.text.GetElapsedValue)
                  70087754    00000014     libc.a : copy_decompress_none.c.obj (.text:decompress:none)
                  70087768    00000008     --HOLE-- [fill = 0]
                  70087770    00000010     app_utils.aer5f : app_utils.oer5f (.text.AppUtils_delay)
                  70087780    0000000e     CanApp.oer5f (.text.CanIf_ControllerBusOff)
                  7008778e    00000002     --HOLE-- [fill = 0]
                  70087790    0000000a     app_utils.aer5f : app_utils_uart.oer5f (.text.getCharacter)
                  7008779a    00000006     --HOLE-- [fill = 0]
                  700877a0    00000008                     : app_utils.oer5f (.text.GetCounterValue)
                  700877a8    00000008     --HOLE-- [fill = 0]
                  700877b0    00000004                     : app_utils.oer5f (.text.AppUtils_SchM_Enter_EXCLUSIVE_AREA_0)
                  700877b4    0000000c     can.aer5f : Can.oer5f (.tramp.Can_1_Int0ISR_Fun.1)
                  700877c0    00000004     app_utils.aer5f : app_utils.oer5f (.text.AppUtils_SchM_Exit_EXCLUSIVE_AREA_0)
                  700877c4    0000000c     can.aer5f : Can.oer5f (.tramp.Can_0_Int1ISR_Fun.1)
                  700877d0    00000004     CanApp.oer5f (.text.SchM_Enter_Can_CAN_EXCLUSIVE_AREA_0)
                  700877d4    0000000c     can.aer5f : Can.oer5f (.tramp.Can_0_Int0ISR_Fun.1)
                  700877e0    00000004     CanApp.oer5f (.text.SchM_Enter_Mcu_MCU_EXCLUSIVE_AREA_0)
                  700877e4    0000000c     --HOLE-- [fill = 0]
                  700877f0    00000004     CanApp.oer5f (.text.SchM_Enter_Port_PORT_EXCLUSIVE_AREA_0)
                  700877f4    0000000c     --HOLE-- [fill = 0]
                  70087800    00000004     CanApp.oer5f (.text.SchM_Exit_Can_CAN_EXCLUSIVE_AREA_0)
                  70087804    0000000c     --HOLE-- [fill = 0]
                  70087810    00000004     CanApp.oer5f (.text.SchM_Exit_Mcu_MCU_EXCLUSIVE_AREA_0)
                  70087814    0000000c     --HOLE-- [fill = 0]
                  70087820    00000004     CanApp.oer5f (.text.SchM_Exit_Port_PORT_EXCLUSIVE_AREA_0)
                  70087824    0000000c     --HOLE-- [fill = 0]
                  70087830    00000004     libclang_rt.builtins.a : aeabi_div0.c.obj (.text.__aeabi_idiv0)
                  70087834    0000000c     --HOLE-- [fill = 0]
                  70087840    00000004                            : aeabi_div0.c.obj (.text.__aeabi_ldiv0)
                  70087844    0000000c     --HOLE-- [fill = 0]
                  70087850    00000002     app_utils.aer5f : app_utils.oer5f (.text.sys_cDabort)
                  70087852    0000000e     --HOLE-- [fill = 0]
                  70087860    00000002                     : app_utils.oer5f (.text.sys_cPabort)
                  70087862    0000000e     --HOLE-- [fill = 0]
                  70087870    00000002                     : app_utils.oer5f (.text.sys_cSwiInt)
                  70087872    0000000e     --HOLE-- [fill = 0]
                  70087880    00000002                     : app_utils.oer5f (.text.sys_cUabort)
                  70087882    0000000e     --HOLE-- [fill = 0]
                  70087890    00000002                     : sys_vim.oer5f (.text.sysphantomInterrupt)
                  70087892    00000102     --HOLE-- [fill = feaa55ef]

.bss       0    70087998    00004998     UNINITIALIZED
                  70087998    00000100     --HOLE--
                  70087a98    000042d8     can.aer5f : Can.oer5f (.bss.gCan_DriverObj)
                  7008bd70    00000400               : Can.oer5f (.bss.CanHtrhMbMapping)
                  7008c170    00000040     (.common:CanRxData)
                  7008c1b0    00000028     (.common:g_sciTransfer)
                  7008c1d8    00000010     port.aer5f : Port.oer5f (.bss.gPortDrvObj)
                  7008c1e8    0000000c     (.common:Pdu)
                  7008c1f4    0000000c     (.common:Pdu1)
                  7008c200    0000000c     (.common:Pdu2)
                  7008c20c    0000000c     (.common:Pdu3)
                  7008c218    00000008     (.common:VersionInfo)
                  7008c220    00000004     (.common:CanIdVal)
                  7008c224    00000004     (.common:eccErrType)
                  7008c228    00000002     (.common:Dem_EventId)
                  7008c22a    00000001     (.common:Dem_EventStatus)
                  7008c22b    00000001     (.common:MainFunc_Execution)
                  7008c22c    00000001     (.common:dlc)
                  7008c22d    00000103     --HOLE--

.stack     0    7008c330    00002000     
                  7008c330    00000004     libc.a : boot_non_cortex_m.S.obj (.stack) [fill = feaa55ef]
                  7008c334    00001ffc     --HOLE-- [fill = feaa55ef]

.sysmem    0    7008e330    00002000     UNINITIALIZED
                  7008e330    00000010     libc.a : memory.c.obj (.sysmem)
                  7008e340    00001ff0     --HOLE--

.rodata    0    70090330    00001dde     
                  70090330    00000200     --HOLE-- [fill = feaa55ef]
                  70090530    00000b98     Port_PBcfg.oer5f (.rodata.PortConfigSet_0_PinConfig)
                  700910c8    00000713     CanApp.oer5f (.rodata.str1.1)
                  700917db    000003be     Port_PBcfg.oer5f (.rodata.str1.1)
                  70091b99    00000003     --HOLE-- [fill = 0]
                  70091b9c    00000180     app_utils.aer5f : app_utils.oer5f (.rodata.gAppUtilsSecHoleAddrList)
                  70091d1c    00000150     Mcu_Cfg.oer5f (.rodata.Mcu_McuClockConfig)
                  70091e6c    00000004     --HOLE-- [fill = 0]
                  70091e70    00000101     libc.a : aeabi_ctype.S.obj (.rodata)
                  70091f71    00000042     app_utils.aer5f : trace.oer5f (.rodata.str1.1)
                  70091fb3    00000001     --HOLE-- [fill = 0]
                  70091fb4    00000040     can.aer5f : mcan.oer5f (.rodata..L__const.MCAN_getDataSize.dataSize)
                  70091ff4    00000031     Dem.oer5f (.rodata.str1.1)
                  70092025    00000022     libc.a : _printfi.c.obj (.rodata.str1.1)
                  70092047    00000001     --HOLE-- [fill = 0]
                  70092048    00000020     Can_PBcfg.oer5f (.rodata.CanConfigSet)
                  70092068    00000020     can.aer5f : mcan.oer5f (.rodata.cst32)
                  70092088    0000001c     Mcu_Cfg.oer5f (.rodata.McuModuleConfiguration)
                  700920a4    00000014     port.aer5f : Port_Platform.oer5f (.rodata.Port_GPIOPortAddr)
                  700920b8    00000010     Port_PBcfg.oer5f (.rodata.PortConfigSet_0)
                  700920c8    00000010     can.aer5f : Can_Mcan.oer5f (.rodata.cst16)
                  700920d8    0000000c     port.aer5f : Port.oer5f (.rodata..L__const.Port_MapConfigToReg.pull_typeselect_map)
                  700920e4    0000000c                : Port.oer5f (.rodata..L__const.Port_MapConfigToReg.slewcontrol_map)
                  700920f0    0000000c     CanApp.oer5f (.rodata..Lswitch.table.CanExample_ExternalTest)
                  700920fc    0000000c     Mcu_Cfg.oer5f (.rodata.Mcu_RamSectionConfig)
                  70092108    00000006     Port_PBcfg.oer5f (.rodata.PortConfigSet_0_DioConfig)

McalConstSection 
*          0    70092110    00001a00     
                  70092110    00001a00     --HOLE-- [fill = feaa55ef]

McalInitSection 
*          0    70093b10    00001a00     UNINITIALIZED
                  70093b10    00001a00     --HOLE--

McalNoInitSection 
*          0    70095510    00001a00     UNINITIALIZED
                  70095510    00001a00     --HOLE--

.data      0    70098910    00001320     UNINITIALIZED
                  70098910    00000100     --HOLE--
                  70098a10    00000bb8     app_utils.aer5f : app_utils.oer5f (.data.AppUtils_printf.tempBuf)
                  700995c8    0000045c     Can_PBcfg.oer5f (.data:CAN_CONFIG_SECTION)
                  70099a24    00000048     CanApp.oer5f (.data.Mcu_RamConfig)
                  70099a6c    00000040     CanApp.oer5f (.data.data)
                  70099aac    0000003c     CanApp.oer5f (.data.gCanAppMcuClockConfig)
                  70099ae8    0000001c     CanApp.oer5f (.data.Mcu_Config)
                  70099b04    00000008     app_utils.aer5f : sys_vim.oer5f (.data.gDrvVim_Stats)
                  70099b0c    00000005     mcu.aer5f : Mcu.oer5f (.data:MCU_DATA_INIT_UNSPECIFIED_SECTION)
                  70099b11    00000001     CanApp.oer5f (.data.CanIf_ControllerModeIndication.controller)
                  70099b12    00000001     can.aer5f : Can.oer5f (.data:CAN_DATA_INIT_UNSPECIFIED_SECTION)
                  70099b13    00000001     --HOLE--
                  70099b14    00000004     CanApp.oer5f (.data.CanExampleFxnTbl)
                  70099b18    00000004     CanApp.oer5f (.data.CanIf_TxConfirmationCount)
                  70099b1c    00000004     libc.a : aeabi_portable.c.obj (.data.__aeabi_errno)
                  70099b20    00000004     CanApp.oer5f (.data.eccErrCnt)
                  70099b24    00000004     CanApp.oer5f (.data.gTestPassed)
                  70099b28    00000004     CanApp.oer5f (.data.msgCounter1)
                  70099b2c    00000004     Port_PBcfg.oer5f (.data:PORT_CONFIG_SECTION)
                  70099b30    00000100     --HOLE--

.const     0    70099c30    00000200     
                  70099c30    00000200     --HOLE-- [fill = feaa55ef]

.cinit     0    70099e30    000004b4     
                  70099e30    00000491     (.cinit..data.load) [load image, compression = rle]
                  7009a2c1    0000000b     (.cinit..bss.load) [load image, compression = rle]
                  7009a2cc    00000008     (__TI_handler_table)
                  7009a2d4    00000010     (__TI_cinit_table)

McalTextSection 
*          0    70096f10    00001a00     
                  70096f10    00001a00     --HOLE-- [fill = feaa55ef]

__llvm_prf_cnts 
*          0    70080000    00000000     UNINITIALIZED

MODULE SUMMARY

       Module                       code    ro data   rw data
       ------                       ----    -------   -------
    D:\TI_SITARA\MCAL_AM263x_00.09.00_03\mcal\binary\can_app\obj\am263\r5f\release\
       CanApp.oer5f                 2006    1823      375    
       Port_PBcfg.oer5f             0       3948      4      
       Can_PBcfg.oer5f              0       32        1116   
       sys_startup.oer5f            992     0         0      
       Mcu_Cfg.oer5f                0       376       0      
       Dem.oer5f                    44      49        3      
       sys_intvecs.oer5f            56      0         0      
    +--+----------------------------+-------+---------+---------+
       Total:                       3098    6228      1498   
                                                             
    C:\ti\ccs1110\ccs\tools\compiler\ti-cgt-armllvm_1.3.0.LTS\lib\armv7r-ti-none-eabihf/c/libc.a
       _printfi.c.obj               6212    34        0      
       s_scalbn.c.obj               320     0         0      
       aeabi_ctype.S.obj            0       257       0      
       vsnprintf.c.obj              236     0         0      
       copy_decompress_rle.c.obj    192     0         0      
       _ltoa.c.obj                  136     0         0      
       s_frexp.c.obj                124     0         0      
       atoi.c.obj                   108     0         0      
       autoinit.c.obj               92      0         0      
       boot_non_cortex_m.S.obj      84      0         0      
       memccpy.c.obj                72      0         0      
       args_main.c.obj              32      0         0      
       wcslen.c.obj                 32      0         0      
       copy_decompress_none.c.obj   20      0         0      
       aeabi_portable.c.obj         12      0         4      
       exit.c.obj                   8       0         0      
       pre_init.c.obj               8       0         0      
       mpu_init.c.obj               4       0         0      
    +--+----------------------------+-------+---------+---------+
       Total:                       7692    291       4      
                                                             
    C:\ti\ccs1110\ccs\tools\compiler\ti-cgt-armllvm_1.3.0.LTS\lib\armv7r-ti-none-eabihf/c/libsysbm.a
       memcpy32.S.obj               28      0         0      
       memset32.S.obj               24      0         0      
    +--+----------------------------+-------+---------+---------+
       Total:                       52      0         0      
                                                             
    C:\ti\ccs1110\ccs\tools\compiler\ti-cgt-armllvm_1.3.0.LTS\lib\clang/12.0.1/lib/armv7r-ti-none-eabihf/libclang_rt.builtins.a
       udivsi3.S.obj                464     0         0      
       udivmoddi4.S.obj             280     0         0      
       divsi3.S.obj                 44      0         0      
       aeabi_uldivmod.S.obj         36      0         0      
       aeabi_memset.S.obj           28      0         0      
       aeabi_div0.c.obj             8       0         0      
       aeabi_memcpy.S.obj           4       0         0      
    +--+----------------------------+-------+---------+---------+
       Total:                       864     0         0      
                                                             
    D:/TI_SITARA/MCAL_AM263x_00.09.00_03/mcal/binary/Can/lib/am263/r5f/release/can.aer5f
       Can.oer5f                    2990    0         18137  
       Can_Mcan.oer5f               4574    16        0      
       mcan.oer5f                   3160    96        0      
       Can_Priv.oer5f               612     0         0      
       Can_Irq.oer5f                116     0         0      
    +--+----------------------------+-------+---------+---------+
       Total:                       11452   112       18137  
                                                             
    D:/TI_SITARA/MCAL_AM263x_00.09.00_03/mcal/binary/Mcu/lib/am263/r5f/release/mcu.aer5f
       Mcu_Platform.oer5f           2742    0         0      
       Mcu.oer5f                    1112    0         5      
    +--+----------------------------+-------+---------+---------+
       Total:                       3854    0         5      
                                                             
    D:/TI_SITARA/MCAL_AM263x_00.09.00_03/mcal/binary/Port/lib/am263/r5f/release/port.aer5f
       Port.oer5f                   1028    24        16     
       Port_Platform.oer5f          748     20        0      
    +--+----------------------------+-------+---------+---------+
       Total:                       1776    44        16     
                                                             
    D:/TI_SITARA/MCAL_AM263x_00.09.00_03/mcal/binary/examples/Utils/lib/am263/r5f/release/app_utils.aer5f
       app_utils.oer5f              258     384       3000   
       sys_vim.oer5f                548     0         8      
       sci.oer5f                    446     0         40     
       sys_core.oer5f               366     0         0      
       trace.oer5f                  168     66        0      
       app_utils_uart.oer5f         86      0         0      
    +--+----------------------------+-------+---------+---------+
       Total:                       1872    450       3048   
                                                             
       Heap:                        0       0         8192   
       Stack:                       0       0         8192   
       Linker Generated:            0       1204      0      
    +--+----------------------------+-------+---------+---------+
       Grand Total:                 30660   8329      39092  


LINKER GENERATED COPY TABLES

__TI_cinit_table @ 7009a2d4 records: 2, size/record: 8, table size: 16
	.data: load addr=70099e30, load size=00000491 bytes, run addr=70098910, run size=00001320 bytes, compression=rle
	.bss: load addr=7009a2c1, load size=0000000b bytes, run addr=70087998, run size=00004998 bytes, compression=rle


LINKER GENERATED HANDLER TABLE

__TI_handler_table @ 7009a2cc records: 2, size/record: 4, table size: 8
	index: 0, handler: __TI_decompress_rle24
	index: 1, handler: __TI_decompress_none

VENEERS

callee name               veneer name
   callee addr  veneer addr  call addr  call info
--------------  -----------  ---------  ----------------
main                      $Ven$AT$L$PI$$main
   70086141     70086dc4     70087608   libc.a : args_main.c.obj (.text._args_main)
Can_3_Int1ISR_Fun         $Ven$AT$L$PI$$Can_3_Int1ISR_Fun
   70085e91     700870f4     70086dc0   can.aer5f : Can_Irq.oer5f (.text:CAN_ISR_TEXT_SECTION)
Can_3_Int0ISR_Fun         $Ven$AT$L$PI$$Can_3_Int0ISR_Fun
   70085e61     70087264     70086db0   can.aer5f : Can_Irq.oer5f (.text:CAN_ISR_TEXT_SECTION)
Can_2_Int1ISR_Fun         $Ven$AT$L$PI$$Can_2_Int1ISR_Fun
   70085e51     70087304     70086da0   can.aer5f : Can_Irq.oer5f (.text:CAN_ISR_TEXT_SECTION)
Can_2_Int0ISR_Fun         $Ven$AT$L$PI$$Can_2_Int0ISR_Fun
   70085e21     70087354     70086d90   can.aer5f : Can_Irq.oer5f (.text:CAN_ISR_TEXT_SECTION)
Can_1_Int1ISR_Fun         $Ven$AT$L$PI$$Can_1_Int1ISR_Fun
   70085e11     700876f4     70086d80   can.aer5f : Can_Irq.oer5f (.text:CAN_ISR_TEXT_SECTION)
Can_1_Int0ISR_Fun         $Ven$AT$L$PI$$Can_1_Int0ISR_Fun
   70085de1     700877b4     70086d70   can.aer5f : Can_Irq.oer5f (.text:CAN_ISR_TEXT_SECTION)
Can_0_Int1ISR_Fun         $Ven$AT$L$PI$$Can_0_Int1ISR_Fun
   70085dd1     700877c4     70086d60   can.aer5f : Can_Irq.oer5f (.text:CAN_ISR_TEXT_SECTION)
Can_0_Int0ISR_Fun         $Ven$AT$L$PI$$Can_0_Int0ISR_Fun
   70085da1     700877d4     70086d50   can.aer5f : Can_Irq.oer5f (.text:CAN_ISR_TEXT_SECTION)

[9 trampolines]
[9 trampoline calls]


FAR CALL TRAMPOLINES

callee name               trampoline name
   callee addr  tramp addr   call addr  call info
--------------  -----------  ---------  ----------------
_sysResetEntry_           $Tramp$AA$L$PI$$_sysResetEntry_
   700851f8     00000038     00000000   sys_intvecs.oer5f (.intvecs)
_sysUndefEntry_           $Tramp$AA$L$PI$$_sysUndefEntry_
   70085208     00000040     00000004   sys_intvecs.oer5f (.intvecs)
_sysSvcEntry_             $Tramp$AA$L$PI$$_sysSvcEntry_
   7008521c     00000048     00000008   sys_intvecs.oer5f (.intvecs)
_sysPrefetchEntry_        $Tramp$AA$L$PI$$_sysPrefetchEntry_
   70085230     00000050     0000000c   sys_intvecs.oer5f (.intvecs)
_sysDAbortEntry_          $Tramp$AA$L$PI$$_sysDAbortEntry_
   70085244     00000058     00000010   sys_intvecs.oer5f (.intvecs)
_sysIrqEntry_             $Tramp$AA$L$PI$$_sysIrqEntry_
   70085258     00000060     00000018   sys_intvecs.oer5f (.intvecs)

[6 trampolines]
[6 trampoline calls]


GLOBAL SYMBOLS: SORTED ALPHABETICALLY BY Name 

address   name                                 
-------   ----                                 
700877b1  AppUtils_SchM_Enter_EXCLUSIVE_AREA_0 
700877c1  AppUtils_SchM_Exit_EXCLUSIVE_AREA_0  
70087361  AppUtils_defaultInit                 
70087771  AppUtils_delay                       
70087631  AppUtils_getChar                     
700873e1  AppUtils_getStackUsage               
700873a1  AppUtils_printf                      
700838c8  C$$EXIT                              
70085300  CSL_armR5EnableIrqFiq                
70085320  CSL_armR5IntrEnableFiq               
70085340  CSL_armR5IntrEnableIrq               
70085360  CSL_armR5IntrEnableVic               
70092048  CanConfigSet                         
70099b14  CanExampleFxnTbl                     
7008bd70  CanHtrhMbMapping                     
7008c220  CanIdVal                             
70087781  CanIf_ControllerBusOff               
700875b1  CanIf_ControllerModeIndication       
70086dd1  CanIf_RxIndication                   
70087651  CanIf_TxConfirmation                 
7008c170  CanRxData                            
70086d50  Can_0_Int0ISR                        
70085da1  Can_0_Int0ISR_Fun                    
70086d60  Can_0_Int1ISR                        
70085dd1  Can_0_Int1ISR_Fun                    
70086d70  Can_1_Int0ISR                        
70085de1  Can_1_Int0ISR_Fun                    
70086d80  Can_1_Int1ISR                        
70085e11  Can_1_Int1ISR_Fun                    
70086d90  Can_2_Int0ISR                        
70085e21  Can_2_Int0ISR_Fun                    
70086da0  Can_2_Int1ISR                        
70085e51  Can_2_Int1ISR_Fun                    
70086db0  Can_3_Int0ISR                        
70085e61  Can_3_Int0ISR_Fun                    
70086dc0  Can_3_Int1ISR                        
70085e91  Can_3_Int1ISR_Fun                    
70083ef1  Can_ChangeBaudrate                   
70083e61  Can_CheckBaudrate                    
70083e11  Can_CheckWakeup                      
700841a1  Can_DeInit                           
70083c91  Can_DisableControllerInterrupts      
70083d21  Can_EnableControllerInterrupts       
70085ea1  Can_GetControllerErrorState          
70085f11  Can_GetControllerMode                
70083b21  Can_GetVersionInfo                   
70083951  Can_Init                             
700840b1  Can_MainFunction_BusOff              
70085ae1  Can_MainFunction_BusOffProcess       
70084111  Can_MainFunction_Mode                
70085af1  Can_MainFunction_ModeProcess         
70084161  Can_MainFunction_Read                
70085b01  Can_MainFunction_ReadProcess         
70084061  Can_MainFunction_Wakeup              
70085ad1  Can_MainFunction_WakeupProcess       
70083d81  Can_MainFunction_Write               
70083fc1  Can_SetBaudrate                      
700838d1  Can_SetControllerMode                
70083b51  Can_Write                            
70085b61  Can_hwDeInit                         
70085ab1  Can_hwUnitChangeBaudrate             
70085aa1  Can_hwUnitCheckWakeup                
70085901  Can_hwUnitConfig                     
70085a71  Can_hwUnitDisableInterrupts          
70085a81  Can_hwUnitEnableInterrupts           
70085ac1  Can_hwUnitSetBaudrate                
70085a01  Can_hwUnitSleep                      
70085991  Can_hwUnitStart                      
700859c1  Can_hwUnitStop                       
70085b51  Can_hwUnitTestLoopBackModeDisable    
70085b41  Can_hwUnitTestLoopBackModeEnable     
70085a91  Can_hwUnitTxDonePolling              
70080c11  Can_mcanChangeBaudrate               
70080d11  Can_mcanCheckWakeup                  
700802b1  Can_mcanConfig                       
70080101  Can_mcanConfigController             
70080ca1  Can_mcanDisableInterrupts            
70080cd1  Can_mcanEnableInterrupts             
70080911  Can_mcanGetProtocolStatus            
700812b1  Can_mcanHwDeInit                     
70080231  Can_mcanInit                         
70080411  Can_mcanInitInterrupt                
70080b41  Can_mcanMsgRAMConfig                 
70080941  Can_mcanMsgRAMConfigInit             
70081181  Can_mcanProcessISR                   
70081271  Can_mcanProcessISRRx                 
70081211  Can_mcanProcessISRTx                 
70080f31  Can_mcanReadRxBuff                   
70081061  Can_mcanReadRxFIFO                   
70080c41  Can_mcanSetBaudrate                  
70080191  Can_mcanSetUpController              
70080381  Can_mcanSetUpMSGRAM                  
700809c1  Can_mcanSetUpRxMailbox               
70080ac1  Can_mcanSetUpTxMailbox               
700805c1  Can_mcanSleep                        
70080441  Can_mcanStart                        
700804c1  Can_mcanStop                         
700806f1  Can_mcanTestLoopBackModeDisable      
70080641  Can_mcanTestLoopBackModeEnable       
70080d31  Can_mcanTxDonePolling                
70085911  Can_mcanWkUp                         
700807a1  Can_mcanWriteGetFreeMsgObj           
70080841  Can_mcanWriteTxMailbox               
70080e21  Can_mcan_BusOffProcess               
70080e71  Can_mcan_ModeProcess                 
70080ef1  Can_mcan_ReadProcess                 
70080de1  Can_mcan_WakeupProcess               
70085a61  Can_writeGetFreeMsgObj               
70085a41  Can_writeTxMailbox                   
7008c228  Dem_EventId                          
7008c22a  Dem_EventStatus                      
70087701  Dem_ReportErrorStatus                
700874d1  Dem_SetEventStatus                   
700875d1  Det_ReportError                      
70087721  Enable_Uart                          
70087211  GT_trace0                            
70087161  GT_trace1                            
700877a1  GetCounterValue                      
70087741  GetElapsedValue                      
70082c01  MCAN_addClockStopRequest             
70082991  MCAN_addExtMsgIDFilter               
70082961  MCAN_addStdMsgIDFilter               
70082b11  MCAN_clearIntrStatus                 
70082841  MCAN_clearNewDataStatus              
70082301  MCAN_config                          
70082c51  MCAN_eccClearErrorStatus             
700823d1  MCAN_eccConfig                       
70082d31  MCAN_eccEnableIntr                   
70082c21  MCAN_eccGetErrorStatus               
70082cf1  MCAN_eccWriteEOI                     
70082a91  MCAN_enableIntr                      
70082ad1  MCAN_enableIntrLine                  
70082d81  MCAN_getBitTime                      
70082d71  MCAN_getClkStopAck                   
70082b01  MCAN_getIntrStatus                   
70082821  MCAN_getNewDataStatus                
700821f1  MCAN_getOpMode                       
70082a41  MCAN_getProtocolStatus               
70082b21  MCAN_getRxFIFOStatus                 
70082b81  MCAN_getTxBufReqPend                 
70082bc1  MCAN_getTxBufTransmissionStatus      
70082201  MCAN_init                            
700821c1  MCAN_isInReset                       
700821d1  MCAN_isMemInitDone                   
700829c1  MCAN_lpbkModeEnable                  
700824f1  MCAN_msgRAMConfig                    
70082861  MCAN_readMsgRam                      
700821b1  MCAN_reset                           
70082ab1  MCAN_selectIntrLine                  
70082411  MCAN_setBitTime                      
70082dd1  MCAN_setExtIDAndMask                 
700821e1  MCAN_setOpMode                       
700827d1  MCAN_txBufAddReq                     
70082b91  MCAN_txBufCancellationReq            
70082bd1  MCAN_txBufCancellationStatus         
70082be1  MCAN_txBufTransIntrEnable            
700826e1  MCAN_writeMsgRam                     
70082b51  MCAN_writeRxFIFOAck                  
70083871  MMR_unlock                           
7008c22b  MainFunc_Execution                   
70092088  McuModuleConfiguration               
70083721  Mcu_ClockSetSourceCPSW               
700836d1  Mcu_ClockSetSourceCPTS               
70082eb1  Mcu_ClockSetSourceCR5                
700834a1  Mcu_ClockSetSourceI2C                
70082f01  Mcu_ClockSetSourceMCAN0              
70082f51  Mcu_ClockSetSourceMCAN1              
70082fa1  Mcu_ClockSetSourceMCAN2              
70082ff1  Mcu_ClockSetSourceMCAN3              
70083311  Mcu_ClockSetSourceMCSPI0             
70083361  Mcu_ClockSetSourceMCSPI1             
700833b1  Mcu_ClockSetSourceMCSPI2             
70083401  Mcu_ClockSetSourceMCSPI3             
70083451  Mcu_ClockSetSourceMCSPI4             
70083811  Mcu_ClockSetSourceMII100Clk          
70083831  Mcu_ClockSetSourceMII10Clk           
70083771  Mcu_ClockSetSourceMcuClkout          
700837c1  Mcu_ClockSetSourcePmicClkout         
700832c1  Mcu_ClockSetSourceQSPI               
70083851  Mcu_ClockSetSourceRGMIClk            
70083041  Mcu_ClockSetSourceRTI0               
70083091  Mcu_ClockSetSourceRTI1               
700830e1  Mcu_ClockSetSourceRTI2               
70083131  Mcu_ClockSetSourceRTI3               
700834f1  Mcu_ClockSetSourceSCI0               
70083541  Mcu_ClockSetSourceSCI1               
70083591  Mcu_ClockSetSourceSCI2               
700835e1  Mcu_ClockSetSourceSCI3               
70083631  Mcu_ClockSetSourceSCI4               
70083681  Mcu_ClockSetSourceSCI5               
70083181  Mcu_ClockSetSourceWDT0               
700831d1  Mcu_ClockSetSourceWDT1               
70083221  Mcu_ClockSetSourceWDT2               
70083271  Mcu_ClockSetSourceWDT3               
70099ae8  Mcu_Config                           
70084bb1  Mcu_DeInit                           
70082e91  Mcu_GetPlatformRawResetReason        
70082e31  Mcu_GetPlatformResetReason           
70084a21  Mcu_GetPllStatus                     
70084b01  Mcu_GetRamState                      
70084ac1  Mcu_GetResetRawValue                 
70084a51  Mcu_GetResetReason                   
70084771  Mcu_GetVersionInfo                   
700847a1  Mcu_Init                             
70084811  Mcu_InitClock                        
700849a1  Mcu_InitRamSection                   
70084b41  Mcu_PerformReset                     
70082e11  Mcu_PerformSoftSysReset              
70099a24  Mcu_RamConfig                        
70084b81  Mcu_RegisterReadback                 
70084a91  Mcu_SetMode                          
70083891  Mcu_unlockMMR                        
7008c1e8  Pdu                                  
7008c1f4  Pdu1                                 
7008c200  Pdu2                                 
7008c20c  Pdu3                                 
700920b8  PortConfigSet_0                      
70099b2c  PortConfigSet_0_pt                   
70085471  Port_ConfigOverrideCtrl              
70085511  Port_ConfigPullInhibitEnable         
700854d1  Port_ConfigPulls                     
700854f1  Port_ConfigSlew                      
70084e61  Port_ConfigurePad                    
70085541  Port_ConfigurePadCore                
70084f91  Port_DeInit                          
70085401  Port_GPIOEdgTrigConfigure            
700853f1  Port_GPIOInit                        
70085461  Port_GPIOIntConfigure                
700853d1  Port_GPIOPortInit                    
70085641  Port_GPIOSetBit                      
700853c1  Port_GetGPIOPortAddr                 
70084f01  Port_GetVersionInfo                  
70084bd1  Port_Init                            
700853b1  Port_LockPadConfig                   
70084f21  Port_MapConfigToReg                  
70085601  Port_ReadMuxMode                     
70084da1  Port_RefreshPortDirection            
700854c1  Port_SelectFunc                      
70085661  Port_SetDirection                    
70084cd1  Port_SetPinDirection                 
70084e81  Port_SetPinMode                      
70085391  Port_UnlockPadConfig                 
70085531  Port_resetPadConfig                  
700877d1  SchM_Enter_Can_CAN_EXCLUSIVE_AREA_0  
700877e1  SchM_Enter_Mcu_MCU_EXCLUSIVE_AREA_0  
700877f1  SchM_Enter_Port_PORT_EXCLUSIVE_AREA_0
70087801  SchM_Exit_Can_CAN_EXCLUSIVE_AREA_0   
70087811  SchM_Exit_Mcu_MCU_EXCLUSIVE_AREA_0   
70087821  SchM_Exit_Port_PORT_EXCLUSIVE_AREA_0 
70087688  TI_memcpy_small                      
700876dc  TI_memset_small                      
7008c218  VersionInfo                          
00001000  __ABORT_STACK_SIZE                   
00001000  __FIQ_STACK_SIZE                     
00001000  __IRQ_STACK_SIZE                     
7008e330  __STACK_END                          
00002000  __STACK_SIZE                         
00001000  __SVC_STACK_SIZE                     
00002000  __SYSMEM_SIZE                        
7009a2d4  __TI_CINIT_Base                      
7009a2e4  __TI_CINIT_Limit                     
7009a2e4  __TI_CINIT_Warm                      
7009a2cc  __TI_Handler_Table_Base              
7009a2d4  __TI_Handler_Table_Limit             
70086fe8  __TI_auto_init_nobinit_nopinit       
70087754  __TI_decompress_none                 
70084bc8  __TI_decompress_rle24                
70086b48  __TI_ltoa                            
ffffffff  __TI_pprof_out_hndl                  
700812e0  __TI_printfi                         
ffffffff  __TI_prof_data_size                  
ffffffff  __TI_prof_data_start                 
00000000  __TI_static_base__                   
00001000  __UND_STACK_SIZE                     
70091e70  __aeabi_ctype_table_                 
70091e70  __aeabi_ctype_table_C                
70099b1c  __aeabi_errno                        
70085384  __aeabi_errno_addr                   
70087500  __aeabi_idiv                         
70087830  __aeabi_idiv0                        
70087840  __aeabi_ldiv0                        
700876b4  __aeabi_memclr                       
700876b4  __aeabi_memclr4                      
700876b4  __aeabi_memclr8                      
700858f8  __aeabi_memcpy                       
700858f8  __aeabi_memcpy4                      
700858f8  __aeabi_memcpy8                      
700876a4  __aeabi_memset                       
700876a4  __aeabi_memset4                      
700876a4  __aeabi_memset8                      
70085f70  __aeabi_uidiv                        
70087584  __aeabi_uldivmod                     
ffffffff  __binit__                            
UNDEFED   __c_args__                           
70087500  __divsi3                             
70093510  __linker_adc_const_end               
70093310  __linker_adc_const_start             
70094f10  __linker_adc_init_end                
70094d10  __linker_adc_init_start              
70096910  __linker_adc_no_init_end             
70096710  __linker_adc_no_init_start           
70098310  __linker_adc_text_end                
70098110  __linker_adc_text_start              
7008c330  __linker_bss_end                     
70087998  __linker_bss_start                   
70093110  __linker_can_const_end               
70092f10  __linker_can_const_start             
70094b10  __linker_can_init_end                
70094910  __linker_can_init_start              
70096510  __linker_can_no_init_end             
70096310  __linker_can_no_init_start           
70097f10  __linker_can_text_end                
70097d10  __linker_can_text_start              
70092f10  __linker_cdd_const_end               
70092d10  __linker_cdd_const_start             
70094910  __linker_cdd_init_end                
70094710  __linker_cdd_init_start              
70096310  __linker_cdd_no_init_end             
70096110  __linker_cdd_no_init_start           
70097d10  __linker_cdd_text_end                
70097b10  __linker_cdd_text_start              
70099e30  __linker_const_end                   
70099c30  __linker_const_start                 
70099c30  __linker_data_end                    
70098910  __linker_data_start                  
70092310  __linker_dio_const_end               
70092110  __linker_dio_const_start             
70093d10  __linker_dio_init_end                
70093b10  __linker_dio_init_start              
70095710  __linker_dio_no_init_end             
70095510  __linker_dio_no_init_start           
70097110  __linker_dio_text_end                
70096f10  __linker_dio_text_start              
70093710  __linker_eth_const_end               
70093510  __linker_eth_const_start             
70095110  __linker_eth_init_end                
70094f10  __linker_eth_init_start              
70096b10  __linker_eth_no_init_end             
70096910  __linker_eth_no_init_start           
70098510  __linker_eth_text_end                
70098310  __linker_eth_text_start              
70093910  __linker_ethtrcv_const_end           
70093710  __linker_ethtrcv_const_start         
70095310  __linker_ethtrcv_init_end            
70095110  __linker_ethtrcv_init_start          
70096d10  __linker_ethtrcv_no_init_end         
70096b10  __linker_ethtrcv_no_init_start       
70098710  __linker_ethtrcv_text_end            
70098510  __linker_ethtrcv_text_start          
70093b10  __linker_fls_const_end               
70093910  __linker_fls_const_start             
70095510  __linker_fls_init_end                
70095310  __linker_fls_init_start              
70096f10  __linker_fls_no_init_end             
70096d10  __linker_fls_no_init_start           
70098910  __linker_fls_text_end                
70098710  __linker_fls_text_start              
70092510  __linker_gpt_const_end               
70092310  __linker_gpt_const_start             
70093f10  __linker_gpt_init_end                
70093d10  __linker_gpt_init_start              
70095910  __linker_gpt_no_init_end             
70095710  __linker_gpt_no_init_start           
70097310  __linker_gpt_text_end                
70097110  __linker_gpt_text_start              
70092710  __linker_mcu_const_end               
70092510  __linker_mcu_const_start             
70094110  __linker_mcu_init_end                
70093f10  __linker_mcu_init_start              
70095b10  __linker_mcu_no_init_end             
70095910  __linker_mcu_no_init_start           
70097510  __linker_mcu_text_end                
70097310  __linker_mcu_text_start              
70092910  __linker_port_const_end              
70092710  __linker_port_const_start            
70094310  __linker_port_init_end               
70094110  __linker_port_init_start             
70095d10  __linker_port_no_init_end            
70095b10  __linker_port_no_init_start          
70097710  __linker_port_text_end               
70097510  __linker_port_text_start             
70093310  __linker_pwm_const_end               
70093110  __linker_pwm_const_start             
70094d10  __linker_pwm_init_end                
70094b10  __linker_pwm_init_start              
70096710  __linker_pwm_no_init_end             
70096510  __linker_pwm_no_init_start           
70098110  __linker_pwm_text_end                
70097f10  __linker_pwm_text_start              
70090530  __linker_rodata_end                  
70090330  __linker_rodata_start                
70092d10  __linker_spi_const_end               
70092b10  __linker_spi_const_start             
70094710  __linker_spi_init_end                
70094510  __linker_spi_init_start              
70096110  __linker_spi_no_init_end             
70095f10  __linker_spi_no_init_start           
70097b10  __linker_spi_text_end                
70097910  __linker_spi_text_start              
70087994  __linker_text_end                    
70080000  __linker_text_start                  
70092b10  __linker_wdg_const_end               
70092910  __linker_wdg_const_start             
70094510  __linker_wdg_init_end                
70094310  __linker_wdg_init_start              
70095f10  __linker_wdg_no_init_end             
70095d10  __linker_wdg_no_init_start           
70097910  __linker_wdg_text_end                
70097710  __linker_wdg_text_start              
7008567c  __mpu_init                           
7008c330  __stack                              
70080000  __start___llvm_prf_cnts              
70080000  __stop___llvm_prf_cnts               
700867e8  __udivmoddi4                         
70085f70  __udivsi3                            
700875f0  _args_main                           
700871b8  _c_int00                             
00000000  _c_int000                            
700863e9  _coreClearAuxiliaryDataFault_        
70086401  _coreClearAuxiliaryInstructionFault_ 
700863b9  _coreClearDataFaultAddress_          
70086389  _coreClearDataFault_                 
700863d1  _coreClearInstructionFaultAddress_   
700863a1  _coreClearInstructionFault_          
700862fb  _coreDisableEventBusExport_          
70086327  _coreDisableRamEcc_                  
70086357  _coreDisableTCMAEcc_                 
700862e5  _coreEnableEventBusExport_           
7008636d  _coreEnableIrqVicOffset_             
70086311  _coreEnableRamEcc_                   
7008633d  _coreEnableTCMAEcc_                  
700862cf  _coreEnableVfp_                      
700863e3  _coreGetAuxiliaryDataFault_          
700863fb  _coreGetAuxiliaryInstructionFault_   
700863b3  _coreGetDataFaultAddress_            
70086383  _coreGetDataFault_                   
700863cb  _coreGetInstructionFaultAddress_     
7008639b  _coreGetInstructionFault_            
70086417  _disable_FIQ_interrupt_              
7008641b  _disable_IRQ_interrupt_              
70086413  _disable_interrupt_                  
7008641f  _enable_interrupt_                   
700851a8  _generateNERROR_                     
700862bd  _getCPSRValue_                       
700862c3  _gotoCPUIdle_                        
7008517c  _meminit_                            
70085064  _pbistTCMB_                          
70085244  _sysDAbortEntry_                     
70086423  _sysDelay_                           
0000001c  _sysFiqEntry_                        
70085258  _sysIrqEntry_                        
70085204  _sysLoop_                            
70085230  _sysPrefetchEntry_                   
70085004  _sysResetCauseHandler_               
700851f8  _sysResetEntry_                      
7008521c  _sysSvcEntry_                        
70085208  _sysUndefEntry_                      
7008e330  _sys_memory                          
UNDEFED   _system_post_cinit                   
70082e08  _system_pre_init                     
700838c8  abort                                
70086e3c  atoi                                 
ffffffff  binit                                
7008c330  bss_end                              
70087998  bss_start                            
70099a6c  data                                 
7008c22c  dlc                                  
7008c224  eccErrType                           
70086c58  frexp                                
70086c58  frexpl                               
70099b04  gDrvVim_Stats                        
70099b0c  gMcuDrvObj                           
70099b24  gTestPassed                          
7008c1b0  g_sciTransfer                        
70087791  getCharacter                         
70082ea1  getMultibitValue                     
70086578  ldexp                                
70086578  ldexpl                               
70086141  main                                 
700872bc  memccpy                              
70087421  message                              
70086578  scalbn                               
70086578  scalbnl                              
70086901  sciAInit                             
70087461  sciDisableNotification               
70087311  sciReceive                           
70087101  sciSend                              
700876c1  sciSetBaudrateValue                  
70087851  sys_cDabort                          
70087861  sys_cPabort                          
70087871  sys_cSwiInt                          
70087881  sys_cUabort                          
700852ac  sys_dataAbtDisp                      
70085294  sys_prefAbtDisp                      
700852c4  sys_swiDisp                          
70085278  sys_udefAbtDisp                      
70087891  sysphantomInterrupt                  
00000190  vimFiqDispatcher                     
70086f21  vimInit                              
70087271  vimInterruptsInit                    
00000100  vimIrqDispatcher                     
70086eb1  vimRegisterInterrupt                 
70086f84  vsnprintf                            
70087610  wcslen                               


GLOBAL SYMBOLS: SORTED BY Symbol Address 

address   name                                 
-------   ----                                 
00000000  __TI_static_base__                   
00000000  _c_int000                            
0000001c  _sysFiqEntry_                        
00000100  vimIrqDispatcher                     
00000190  vimFiqDispatcher                     
00001000  __ABORT_STACK_SIZE                   
00001000  __FIQ_STACK_SIZE                     
00001000  __IRQ_STACK_SIZE                     
00001000  __SVC_STACK_SIZE                     
00001000  __UND_STACK_SIZE                     
00002000  __STACK_SIZE                         
00002000  __SYSMEM_SIZE                        
70080000  __linker_text_start                  
70080000  __start___llvm_prf_cnts              
70080000  __stop___llvm_prf_cnts               
70080101  Can_mcanConfigController             
70080191  Can_mcanSetUpController              
70080231  Can_mcanInit                         
700802b1  Can_mcanConfig                       
70080381  Can_mcanSetUpMSGRAM                  
70080411  Can_mcanInitInterrupt                
70080441  Can_mcanStart                        
700804c1  Can_mcanStop                         
700805c1  Can_mcanSleep                        
70080641  Can_mcanTestLoopBackModeEnable       
700806f1  Can_mcanTestLoopBackModeDisable      
700807a1  Can_mcanWriteGetFreeMsgObj           
70080841  Can_mcanWriteTxMailbox               
70080911  Can_mcanGetProtocolStatus            
70080941  Can_mcanMsgRAMConfigInit             
700809c1  Can_mcanSetUpRxMailbox               
70080ac1  Can_mcanSetUpTxMailbox               
70080b41  Can_mcanMsgRAMConfig                 
70080c11  Can_mcanChangeBaudrate               
70080c41  Can_mcanSetBaudrate                  
70080ca1  Can_mcanDisableInterrupts            
70080cd1  Can_mcanEnableInterrupts             
70080d11  Can_mcanCheckWakeup                  
70080d31  Can_mcanTxDonePolling                
70080de1  Can_mcan_WakeupProcess               
70080e21  Can_mcan_BusOffProcess               
70080e71  Can_mcan_ModeProcess                 
70080ef1  Can_mcan_ReadProcess                 
70080f31  Can_mcanReadRxBuff                   
70081061  Can_mcanReadRxFIFO                   
70081181  Can_mcanProcessISR                   
70081211  Can_mcanProcessISRTx                 
70081271  Can_mcanProcessISRRx                 
700812b1  Can_mcanHwDeInit                     
700812e0  __TI_printfi                         
700821b1  MCAN_reset                           
700821c1  MCAN_isInReset                       
700821d1  MCAN_isMemInitDone                   
700821e1  MCAN_setOpMode                       
700821f1  MCAN_getOpMode                       
70082201  MCAN_init                            
70082301  MCAN_config                          
700823d1  MCAN_eccConfig                       
70082411  MCAN_setBitTime                      
700824f1  MCAN_msgRAMConfig                    
700826e1  MCAN_writeMsgRam                     
700827d1  MCAN_txBufAddReq                     
70082821  MCAN_getNewDataStatus                
70082841  MCAN_clearNewDataStatus              
70082861  MCAN_readMsgRam                      
70082961  MCAN_addStdMsgIDFilter               
70082991  MCAN_addExtMsgIDFilter               
700829c1  MCAN_lpbkModeEnable                  
70082a41  MCAN_getProtocolStatus               
70082a91  MCAN_enableIntr                      
70082ab1  MCAN_selectIntrLine                  
70082ad1  MCAN_enableIntrLine                  
70082b01  MCAN_getIntrStatus                   
70082b11  MCAN_clearIntrStatus                 
70082b21  MCAN_getRxFIFOStatus                 
70082b51  MCAN_writeRxFIFOAck                  
70082b81  MCAN_getTxBufReqPend                 
70082b91  MCAN_txBufCancellationReq            
70082bc1  MCAN_getTxBufTransmissionStatus      
70082bd1  MCAN_txBufCancellationStatus         
70082be1  MCAN_txBufTransIntrEnable            
70082c01  MCAN_addClockStopRequest             
70082c21  MCAN_eccGetErrorStatus               
70082c51  MCAN_eccClearErrorStatus             
70082cf1  MCAN_eccWriteEOI                     
70082d31  MCAN_eccEnableIntr                   
70082d71  MCAN_getClkStopAck                   
70082d81  MCAN_getBitTime                      
70082dd1  MCAN_setExtIDAndMask                 
70082e08  _system_pre_init                     
70082e11  Mcu_PerformSoftSysReset              
70082e31  Mcu_GetPlatformResetReason           
70082e91  Mcu_GetPlatformRawResetReason        
70082ea1  getMultibitValue                     
70082eb1  Mcu_ClockSetSourceCR5                
70082f01  Mcu_ClockSetSourceMCAN0              
70082f51  Mcu_ClockSetSourceMCAN1              
70082fa1  Mcu_ClockSetSourceMCAN2              
70082ff1  Mcu_ClockSetSourceMCAN3              
70083041  Mcu_ClockSetSourceRTI0               
70083091  Mcu_ClockSetSourceRTI1               
700830e1  Mcu_ClockSetSourceRTI2               
70083131  Mcu_ClockSetSourceRTI3               
70083181  Mcu_ClockSetSourceWDT0               
700831d1  Mcu_ClockSetSourceWDT1               
70083221  Mcu_ClockSetSourceWDT2               
70083271  Mcu_ClockSetSourceWDT3               
700832c1  Mcu_ClockSetSourceQSPI               
70083311  Mcu_ClockSetSourceMCSPI0             
70083361  Mcu_ClockSetSourceMCSPI1             
700833b1  Mcu_ClockSetSourceMCSPI2             
70083401  Mcu_ClockSetSourceMCSPI3             
70083451  Mcu_ClockSetSourceMCSPI4             
700834a1  Mcu_ClockSetSourceI2C                
700834f1  Mcu_ClockSetSourceSCI0               
70083541  Mcu_ClockSetSourceSCI1               
70083591  Mcu_ClockSetSourceSCI2               
700835e1  Mcu_ClockSetSourceSCI3               
70083631  Mcu_ClockSetSourceSCI4               
70083681  Mcu_ClockSetSourceSCI5               
700836d1  Mcu_ClockSetSourceCPTS               
70083721  Mcu_ClockSetSourceCPSW               
70083771  Mcu_ClockSetSourceMcuClkout          
700837c1  Mcu_ClockSetSourcePmicClkout         
70083811  Mcu_ClockSetSourceMII100Clk          
70083831  Mcu_ClockSetSourceMII10Clk           
70083851  Mcu_ClockSetSourceRGMIClk            
70083871  MMR_unlock                           
70083891  Mcu_unlockMMR                        
700838c8  C$$EXIT                              
700838c8  abort                                
700838d1  Can_SetControllerMode                
70083951  Can_Init                             
70083b21  Can_GetVersionInfo                   
70083b51  Can_Write                            
70083c91  Can_DisableControllerInterrupts      
70083d21  Can_EnableControllerInterrupts       
70083d81  Can_MainFunction_Write               
70083e11  Can_CheckWakeup                      
70083e61  Can_CheckBaudrate                    
70083ef1  Can_ChangeBaudrate                   
70083fc1  Can_SetBaudrate                      
70084061  Can_MainFunction_Wakeup              
700840b1  Can_MainFunction_BusOff              
70084111  Can_MainFunction_Mode                
70084161  Can_MainFunction_Read                
700841a1  Can_DeInit                           
70084771  Mcu_GetVersionInfo                   
700847a1  Mcu_Init                             
70084811  Mcu_InitClock                        
700849a1  Mcu_InitRamSection                   
70084a21  Mcu_GetPllStatus                     
70084a51  Mcu_GetResetReason                   
70084a91  Mcu_SetMode                          
70084ac1  Mcu_GetResetRawValue                 
70084b01  Mcu_GetRamState                      
70084b41  Mcu_PerformReset                     
70084b81  Mcu_RegisterReadback                 
70084bb1  Mcu_DeInit                           
70084bc8  __TI_decompress_rle24                
70084bd1  Port_Init                            
70084cd1  Port_SetPinDirection                 
70084da1  Port_RefreshPortDirection            
70084e61  Port_ConfigurePad                    
70084e81  Port_SetPinMode                      
70084f01  Port_GetVersionInfo                  
70084f21  Port_MapConfigToReg                  
70084f91  Port_DeInit                          
70085004  _sysResetCauseHandler_               
70085064  _pbistTCMB_                          
7008517c  _meminit_                            
700851a8  _generateNERROR_                     
700851f8  _sysResetEntry_                      
70085204  _sysLoop_                            
70085208  _sysUndefEntry_                      
7008521c  _sysSvcEntry_                        
70085230  _sysPrefetchEntry_                   
70085244  _sysDAbortEntry_                     
70085258  _sysIrqEntry_                        
70085278  sys_udefAbtDisp                      
70085294  sys_prefAbtDisp                      
700852ac  sys_dataAbtDisp                      
700852c4  sys_swiDisp                          
70085300  CSL_armR5EnableIrqFiq                
70085320  CSL_armR5IntrEnableFiq               
70085340  CSL_armR5IntrEnableIrq               
70085360  CSL_armR5IntrEnableVic               
70085384  __aeabi_errno_addr                   
70085391  Port_UnlockPadConfig                 
700853b1  Port_LockPadConfig                   
700853c1  Port_GetGPIOPortAddr                 
700853d1  Port_GPIOPortInit                    
700853f1  Port_GPIOInit                        
70085401  Port_GPIOEdgTrigConfigure            
70085461  Port_GPIOIntConfigure                
70085471  Port_ConfigOverrideCtrl              
700854c1  Port_SelectFunc                      
700854d1  Port_ConfigPulls                     
700854f1  Port_ConfigSlew                      
70085511  Port_ConfigPullInhibitEnable         
70085531  Port_resetPadConfig                  
70085541  Port_ConfigurePadCore                
70085601  Port_ReadMuxMode                     
70085641  Port_GPIOSetBit                      
70085661  Port_SetDirection                    
7008567c  __mpu_init                           
700858f8  __aeabi_memcpy                       
700858f8  __aeabi_memcpy4                      
700858f8  __aeabi_memcpy8                      
70085901  Can_hwUnitConfig                     
70085911  Can_mcanWkUp                         
70085991  Can_hwUnitStart                      
700859c1  Can_hwUnitStop                       
70085a01  Can_hwUnitSleep                      
70085a41  Can_writeTxMailbox                   
70085a61  Can_writeGetFreeMsgObj               
70085a71  Can_hwUnitDisableInterrupts          
70085a81  Can_hwUnitEnableInterrupts           
70085a91  Can_hwUnitTxDonePolling              
70085aa1  Can_hwUnitCheckWakeup                
70085ab1  Can_hwUnitChangeBaudrate             
70085ac1  Can_hwUnitSetBaudrate                
70085ad1  Can_MainFunction_WakeupProcess       
70085ae1  Can_MainFunction_BusOffProcess       
70085af1  Can_MainFunction_ModeProcess         
70085b01  Can_MainFunction_ReadProcess         
70085b41  Can_hwUnitTestLoopBackModeEnable     
70085b51  Can_hwUnitTestLoopBackModeDisable    
70085b61  Can_hwDeInit                         
70085da1  Can_0_Int0ISR_Fun                    
70085dd1  Can_0_Int1ISR_Fun                    
70085de1  Can_1_Int0ISR_Fun                    
70085e11  Can_1_Int1ISR_Fun                    
70085e21  Can_2_Int0ISR_Fun                    
70085e51  Can_2_Int1ISR_Fun                    
70085e61  Can_3_Int0ISR_Fun                    
70085e91  Can_3_Int1ISR_Fun                    
70085ea1  Can_GetControllerErrorState          
70085f11  Can_GetControllerMode                
70085f70  __aeabi_uidiv                        
70085f70  __udivsi3                            
70086141  main                                 
700862bd  _getCPSRValue_                       
700862c3  _gotoCPUIdle_                        
700862cf  _coreEnableVfp_                      
700862e5  _coreEnableEventBusExport_           
700862fb  _coreDisableEventBusExport_          
70086311  _coreEnableRamEcc_                   
70086327  _coreDisableRamEcc_                  
7008633d  _coreEnableTCMAEcc_                  
70086357  _coreDisableTCMAEcc_                 
7008636d  _coreEnableIrqVicOffset_             
70086383  _coreGetDataFault_                   
70086389  _coreClearDataFault_                 
7008639b  _coreGetInstructionFault_            
700863a1  _coreClearInstructionFault_          
700863b3  _coreGetDataFaultAddress_            
700863b9  _coreClearDataFaultAddress_          
700863cb  _coreGetInstructionFaultAddress_     
700863d1  _coreClearInstructionFaultAddress_   
700863e3  _coreGetAuxiliaryDataFault_          
700863e9  _coreClearAuxiliaryDataFault_        
700863fb  _coreGetAuxiliaryInstructionFault_   
70086401  _coreClearAuxiliaryInstructionFault_ 
70086413  _disable_interrupt_                  
70086417  _disable_FIQ_interrupt_              
7008641b  _disable_IRQ_interrupt_              
7008641f  _enable_interrupt_                   
70086423  _sysDelay_                           
70086578  ldexp                                
70086578  ldexpl                               
70086578  scalbn                               
70086578  scalbnl                              
700867e8  __udivmoddi4                         
70086901  sciAInit                             
70086b48  __TI_ltoa                            
70086c58  frexp                                
70086c58  frexpl                               
70086d50  Can_0_Int0ISR                        
70086d60  Can_0_Int1ISR                        
70086d70  Can_1_Int0ISR                        
70086d80  Can_1_Int1ISR                        
70086d90  Can_2_Int0ISR                        
70086da0  Can_2_Int1ISR                        
70086db0  Can_3_Int0ISR                        
70086dc0  Can_3_Int1ISR                        
70086dd1  CanIf_RxIndication                   
70086e3c  atoi                                 
70086eb1  vimRegisterInterrupt                 
70086f21  vimInit                              
70086f84  vsnprintf                            
70086fe8  __TI_auto_init_nobinit_nopinit       
70087101  sciSend                              
70087161  GT_trace1                            
700871b8  _c_int00                             
70087211  GT_trace0                            
70087271  vimInterruptsInit                    
700872bc  memccpy                              
70087311  sciReceive                           
70087361  AppUtils_defaultInit                 
700873a1  AppUtils_printf                      
700873e1  AppUtils_getStackUsage               
70087421  message                              
70087461  sciDisableNotification               
700874d1  Dem_SetEventStatus                   
70087500  __aeabi_idiv                         
70087500  __divsi3                             
70087584  __aeabi_uldivmod                     
700875b1  CanIf_ControllerModeIndication       
700875d1  Det_ReportError                      
700875f0  _args_main                           
70087610  wcslen                               
70087631  AppUtils_getChar                     
70087651  CanIf_TxConfirmation                 
70087688  TI_memcpy_small                      
700876a4  __aeabi_memset                       
700876a4  __aeabi_memset4                      
700876a4  __aeabi_memset8                      
700876b4  __aeabi_memclr                       
700876b4  __aeabi_memclr4                      
700876b4  __aeabi_memclr8                      
700876c1  sciSetBaudrateValue                  
700876dc  TI_memset_small                      
70087701  Dem_ReportErrorStatus                
70087721  Enable_Uart                          
70087741  GetElapsedValue                      
70087754  __TI_decompress_none                 
70087771  AppUtils_delay                       
70087781  CanIf_ControllerBusOff               
70087791  getCharacter                         
700877a1  GetCounterValue                      
700877b1  AppUtils_SchM_Enter_EXCLUSIVE_AREA_0 
700877c1  AppUtils_SchM_Exit_EXCLUSIVE_AREA_0  
700877d1  SchM_Enter_Can_CAN_EXCLUSIVE_AREA_0  
700877e1  SchM_Enter_Mcu_MCU_EXCLUSIVE_AREA_0  
700877f1  SchM_Enter_Port_PORT_EXCLUSIVE_AREA_0
70087801  SchM_Exit_Can_CAN_EXCLUSIVE_AREA_0   
70087811  SchM_Exit_Mcu_MCU_EXCLUSIVE_AREA_0   
70087821  SchM_Exit_Port_PORT_EXCLUSIVE_AREA_0 
70087830  __aeabi_idiv0                        
70087840  __aeabi_ldiv0                        
70087851  sys_cDabort                          
70087861  sys_cPabort                          
70087871  sys_cSwiInt                          
70087881  sys_cUabort                          
70087891  sysphantomInterrupt                  
70087994  __linker_text_end                    
70087998  __linker_bss_start                   
70087998  bss_start                            
7008bd70  CanHtrhMbMapping                     
7008c170  CanRxData                            
7008c1b0  g_sciTransfer                        
7008c1e8  Pdu                                  
7008c1f4  Pdu1                                 
7008c200  Pdu2                                 
7008c20c  Pdu3                                 
7008c218  VersionInfo                          
7008c220  CanIdVal                             
7008c224  eccErrType                           
7008c228  Dem_EventId                          
7008c22a  Dem_EventStatus                      
7008c22b  MainFunc_Execution                   
7008c22c  dlc                                  
7008c330  __linker_bss_end                     
7008c330  __stack                              
7008c330  bss_end                              
7008e330  __STACK_END                          
7008e330  _sys_memory                          
70090330  __linker_rodata_start                
70090530  __linker_rodata_end                  
70091e70  __aeabi_ctype_table_                 
70091e70  __aeabi_ctype_table_C                
70092048  CanConfigSet                         
70092088  McuModuleConfiguration               
700920b8  PortConfigSet_0                      
70092110  __linker_dio_const_start             
70092310  __linker_dio_const_end               
70092310  __linker_gpt_const_start             
70092510  __linker_gpt_const_end               
70092510  __linker_mcu_const_start             
70092710  __linker_mcu_const_end               
70092710  __linker_port_const_start            
70092910  __linker_port_const_end              
70092910  __linker_wdg_const_start             
70092b10  __linker_spi_const_start             
70092b10  __linker_wdg_const_end               
70092d10  __linker_cdd_const_start             
70092d10  __linker_spi_const_end               
70092f10  __linker_can_const_start             
70092f10  __linker_cdd_const_end               
70093110  __linker_can_const_end               
70093110  __linker_pwm_const_start             
70093310  __linker_adc_const_start             
70093310  __linker_pwm_const_end               
70093510  __linker_adc_const_end               
70093510  __linker_eth_const_start             
70093710  __linker_eth_const_end               
70093710  __linker_ethtrcv_const_start         
70093910  __linker_ethtrcv_const_end           
70093910  __linker_fls_const_start             
70093b10  __linker_dio_init_start              
70093b10  __linker_fls_const_end               
70093d10  __linker_dio_init_end                
70093d10  __linker_gpt_init_start              
70093f10  __linker_gpt_init_end                
70093f10  __linker_mcu_init_start              
70094110  __linker_mcu_init_end                
70094110  __linker_port_init_start             
70094310  __linker_port_init_end               
70094310  __linker_wdg_init_start              
70094510  __linker_spi_init_start              
70094510  __linker_wdg_init_end                
70094710  __linker_cdd_init_start              
70094710  __linker_spi_init_end                
70094910  __linker_can_init_start              
70094910  __linker_cdd_init_end                
70094b10  __linker_can_init_end                
70094b10  __linker_pwm_init_start              
70094d10  __linker_adc_init_start              
70094d10  __linker_pwm_init_end                
70094f10  __linker_adc_init_end                
70094f10  __linker_eth_init_start              
70095110  __linker_eth_init_end                
70095110  __linker_ethtrcv_init_start          
70095310  __linker_ethtrcv_init_end            
70095310  __linker_fls_init_start              
70095510  __linker_dio_no_init_start           
70095510  __linker_fls_init_end                
70095710  __linker_dio_no_init_end             
70095710  __linker_gpt_no_init_start           
70095910  __linker_gpt_no_init_end             
70095910  __linker_mcu_no_init_start           
70095b10  __linker_mcu_no_init_end             
70095b10  __linker_port_no_init_start          
70095d10  __linker_port_no_init_end            
70095d10  __linker_wdg_no_init_start           
70095f10  __linker_spi_no_init_start           
70095f10  __linker_wdg_no_init_end             
70096110  __linker_cdd_no_init_start           
70096110  __linker_spi_no_init_end             
70096310  __linker_can_no_init_start           
70096310  __linker_cdd_no_init_end             
70096510  __linker_can_no_init_end             
70096510  __linker_pwm_no_init_start           
70096710  __linker_adc_no_init_start           
70096710  __linker_pwm_no_init_end             
70096910  __linker_adc_no_init_end             
70096910  __linker_eth_no_init_start           
70096b10  __linker_eth_no_init_end             
70096b10  __linker_ethtrcv_no_init_start       
70096d10  __linker_ethtrcv_no_init_end         
70096d10  __linker_fls_no_init_start           
70096f10  __linker_dio_text_start              
70096f10  __linker_fls_no_init_end             
70097110  __linker_dio_text_end                
70097110  __linker_gpt_text_start              
70097310  __linker_gpt_text_end                
70097310  __linker_mcu_text_start              
70097510  __linker_mcu_text_end                
70097510  __linker_port_text_start             
70097710  __linker_port_text_end               
70097710  __linker_wdg_text_start              
70097910  __linker_spi_text_start              
70097910  __linker_wdg_text_end                
70097b10  __linker_cdd_text_start              
70097b10  __linker_spi_text_end                
70097d10  __linker_can_text_start              
70097d10  __linker_cdd_text_end                
70097f10  __linker_can_text_end                
70097f10  __linker_pwm_text_start              
70098110  __linker_adc_text_start              
70098110  __linker_pwm_text_end                
70098310  __linker_adc_text_end                
70098310  __linker_eth_text_start              
70098510  __linker_eth_text_end                
70098510  __linker_ethtrcv_text_start          
70098710  __linker_ethtrcv_text_end            
70098710  __linker_fls_text_start              
70098910  __linker_data_start                  
70098910  __linker_fls_text_end                
70099a24  Mcu_RamConfig                        
70099a6c  data                                 
70099ae8  Mcu_Config                           
70099b04  gDrvVim_Stats                        
70099b0c  gMcuDrvObj                           
70099b14  CanExampleFxnTbl                     
70099b1c  __aeabi_errno                        
70099b24  gTestPassed                          
70099b2c  PortConfigSet_0_pt                   
70099c30  __linker_const_start                 
70099c30  __linker_data_end                    
70099e30  __linker_const_end                   
7009a2cc  __TI_Handler_Table_Base              
7009a2d4  __TI_CINIT_Base                      
7009a2d4  __TI_Handler_Table_Limit             
7009a2e4  __TI_CINIT_Limit                     
7009a2e4  __TI_CINIT_Warm                      
ffffffff  __TI_pprof_out_hndl                  
ffffffff  __TI_prof_data_size                  
ffffffff  __TI_prof_data_start                 
ffffffff  __binit__                            
ffffffff  binit                                
UNDEFED   __c_args__                           
UNDEFED   _system_post_cinit                   

[504 symbols]
